:10000000830100308A002428F60003088301CA0017
:100010008B1A0B1D1D280B11F03083120313810066
:10002000AB0AA11C1728AC0A031D1728A115211D16
:100030001D28AD0A031D1D282116031383124A082B
:100040008300F60E760E09002230840048303120FD
:1000500020308400223031208301FA2C04068001F4
:10006000840A0406031D2E28003483120313C800DB
:10007000C91B4328491B4B2849088A004808C80A5D
:100080000319C90A82008313491883174808C80A4C
:10009000840000080800FC34FE34073403340334C1
:1000A000033403340734FE34FC340F341F34383443
:1000B000303430343034303438341F340F3400347A
:1000C00008340C340E34FF34FF3400340034003470
:1000D000003400340034303430343F343F34303472
:1000E0003034003400340C340E3407340334033419
:1000F0008334C334E7347E341C34303438343C34F5
:100100003E343734333431343034303430340C34DA
:100110000E34073403340334C334E734F634BE34C6
:100120001C340C341C3438343034303430343034F3
:1001300039341F340F34FF34FF34C034C034C0347A
:10014000C034C034C034FF34FF34003400340034D1
:10015000003400340034003400343F343F347F3402
:100160007F3463346334633463346334E334C334DB
:10017000833430343034303430343034303430340C
:1001800038341F340F34FC34FE34C73463346334E2
:1001900063346334E334C73486340F341F34383463
:1001A000303430343034303438341F340F34033486
:1001B000033403348334C334E33473343B341F34A3
:1001C0000F343C343E3407340334013400340034FB
:1001D0000034003400341C34BE34F73463346334E8
:1001E00063346334F734BE341C340F341F34393471
:1001F000303430343034303439341F340F343C34FC
:100200007E34E734C334C334C334C334C734FE3418
:10021000FC340C341C343834303430343034303422
:1002200038341F340F34C034C034C034C034C03408
:10023000C034C034C034C034C0340034003400345E
:10024000003400340034003400340034003400340E
:1002500000340034003400340034003400340034FE
:1002600000340034003400340034003400340034EE
:1002700000340034003400340034003400340034DE
:1002800000340034003400340034003400343C3492
:100290003C343C343C34003400340034003400340A
:1002A0000034003400341E343F34333433343F34AC
:1002B0001E34003400340034003400340034003480
:1002C000003400340034F834FC340E340734033482
:1002D0000334033407340E340C3407341F341C3415
:1002E000383430343034303438341C340C348207F1
:1002F000C0347E3441347F34C034383444344434E0
:10030000443438347C340834103408347C340834B1
:10031000083408340834083427344834483448341E
:100320003F3440343834043404347C347C34203456
:10033000103408347C347C34403440347C34C03451
:100340002034543454345434783400340034003479
:10035000003400347F3408341434223441342234DD
:1003600049344934493436343E34413441344134DB
:100370003E347F3445344534453439347F34093490
:100380000934093406347F344834303400347F343F
:100390007F3449344934493436347F3402340434A8
:1003A00002347F34043404347C34043404347C3424
:0803B000143414341434083431
:1005020002308301BE00BE0B842A08001230830130
:10051200BE00BE0B8A2A08008A308301BC00BC0BD5
:10052200902A08009E308301BC00BC0B962A08006A
:100532008301C40086168610612386140800830195
:10054200C000861286106123861408008301BF0052
:100552003E0807394038A0223F087F398038A02A58
:1005620083012B08BD001930BD072B083D02BC00DA
:10057200BC08031908006400B62AF401F50103104F
:10058200F30CF20C031CCC2A7008F4077108031850
:10059200710AF5070310F00DF10D720873040319C7
:1005A2000034C02A8301BE010030A722F830BC000B
:1005B2000130BD00640000309922BC080319BD035C
:1005C200BC033D08803AF00080307002013003190C
:1005D2003C02031C0800DB2A640083120313861505
:1005E200861400008611B12286152130A022C23065
:1005F200A0220730A0221330A0222030A0220930EE
:10060200A022D3220830A0220C30A022BE0100304A
:10061200A72A073083019F0086018501FF308316D8
:100622008500C430860020308B0083128C01831633
:100632008C0107308100F030831281008B17A013E8
:10064200A111A110211021122111080008308301EB
:10065200BC00BD01640005128316051200000000F3
:100662000000051681222011051A20158722031089
:10067200BD0C201D3E2B8030BD078122BC0B2B2BD5
:1006820081223D08080008308301BC00BD016400DE
:1006920006118316061100000000000006158122D3
:1006A200A0100619A01487220310BD0CA01C5B2BFE
:1006B2008030BD078122BC0B482B81223D080800F7
:1006C2008301C50064000830C600C7010612C51FB9
:1006D2006C2B06146D2B061006160310C50DC608EA
:1006E2000319C703C6034708803AF000803070023E
:1006F200013003194602031C0800672B8301BC006A
:10070200C100C2010530BF00C00101308A004108AA
:100712007721BD00BE019922C10A0319C20ABF088E
:100722000319C003BF034008803AF0008030700212
:10073200013003193F020318862B0030992A8301E6
:10074200BC000830BD00A0103C18A0148312031393
:10075200061183160611000000000000000083123B
:10076200A01CB62B83160615B82B831606118722FA
:100772008316061581220310BC0CBD0BA42B812A03
:100782008301BC000830BD0020113C1820158312E3
:10079200031305128316051200000000000000007A
:1007A2008312201DD72B83160516D92B831605120B
:1007B20087228316051681220310BC0CBD0BC52BA4
:1007C200812A83013C08C2003D08C3000A30C000F0
:1007D200C1014308003EC90042084B3E0318C90A42
:1007E2003520BE00BF019922C20A0319C30AC008FC
:0E07F2000319C103C0034108803AF0008030B3
:1008000070020130031940020318EA2B00309922CC
:100810000030992A640083120313A301A2018316F6
:100820000516061583120512061183160512061108
:1008300093228316051606158722A0110619A01506
:10084000831203132012051A20168D22A0120619F6
:10085000A016831203132013051A2017A01A322C96
:10086000A201A20A201B362CA301A30AA01D3A2C28
:100870000230A207201E812A0230A307812A8301A9
:10088000BD003C08BA00BB01BB00BA013D08BA0478
:10089000BB1F5A2C20143B08F1003A08F000F00965
:1008A000F10901307007BA000030031801307107F8
:1008B000BB005B2C20100530F200F3013B08F10077
:1008C0003A08F000BE227408AE007508AF002F0D84
:1008D000AF0CAE0C2F0DAF0CAE0C2F0DAF0CAE0C41
:1008E000A501A401A6012E08B8002F08B9003908F7
:1008F000803AF000803070020A3003193802031C7D
:10090000AC2CF630380739080318390AFF3E803915
:10091000031D8F2CA60AF630B807031CB90326085E
:10092000F000F101F63E71080318710AFF3E8039AC
:10093000031D9D2CA40AF630A6072408F000F1013F
:10094000F63E71080318710AFF3E8039031D772CAB
:10095000A50AF630A407772C3808B6003908B70086
:100960002608B400B5012408B200B3012508B00080
:10097000B101201CBE2C0A30B000B101A508031D36
:100980000800A408031DF02CA608031DE52C390857
:100990003804031DD82C0B30B400B501B200350863
:1009A000B3003208B0003308B100B601B701080047
:1009B000201CDC2C0A30DD2C0B30B200B3010B30D4
:1009C000B000B101B401B5010800201CE92C0A30C7
:1009D000EA2C0B30B200B3010B30B000B1010800BB
:1009E000201CF62C0A30B000B10108000B30B0001A
:1009F000B101080064000A23ED22BE010030A722E5
:100A00000F307F230F307F230F307F230F307F2362
:100A10002D307F2355307F2305307F235A307F23AD
:100A200005307F235F307F232D307F230F307F23DE
:100A30000F307F230F307F230330BE000030A7220A
:100A40000F307F230F307F230F307F230F307F2322
:100A50002D307F2314307F2319307F231E307F23D6
:100A600023307F2328307F232D307F230F307F23B7
:100A70000F307F230F307F238B130A248B17220321
:100A800003195F2E2208023A0319272E8B13CC304C
:100A9000A0238B17A118532D8B134430A0238B1741
:100AA000A114AC01A111A118061D5D2DA11D5D2D84
:100AB0008B13BE30A0238B17A017B122A01F9F2E2F
:100AC0008B134423A7004423A9008B17BC002708DD
:100AD0003F24A111A110A013BE01BE0A0030A7221D
:100AE0001430F200F3013108F1003008F000BE22AA
:100AF0007408BC007508BD00E2231430F200F30155
:100B00003308F1003208F000BE227408BC007508FA
:100B1000BD00E2231430F200F3013508F10034087F
:100B2000F000BE227408BC007508BD00E223A508D1
:100B3000031DA62DA408031DA62DA608031DA62D82
:100B400039083804031DA62DDC30A72DF030BC0079
:100B5000BD01E2231430F200F3013708F10036083A
:100B6000F000BE227408BC007508BD00E22304300A
:100B7000BC000130BD00E2231830BC000130BD00D4
:100B8000E2230230BE000030A7221430F200F3014D
:100B90003108F1003008F000BE220A307407BC00B2
:100BA0000030031801307507BD00E2231430F20055
:100BB000F3013308F1003208F000BE220A30740756
:100BC000BC000030031801307507BD00E22314306B
:100BD000F200F3013508F1003408F000BE220A30BB
:100BE0007407BC000030031801307507BD00E22314
:100BF000A508031D072EA408031D072EA608031D24
:100C0000072E39083804031D072EE630082EFA3067
:100C1000BC00BD01E2231430F200F3013708F100FB
:100C20003608F000BE220A307407BC0000300318FA
:100C300001307507BD00E2230E30BC000130BD005D
:100C4000E2232230BC000130BD00E2239F2EBE0112
:100C5000BE0A0030A7222D307F232D307F232D3078
:100C60007F232D307F232D307F232D307F232D3088
:100C70007F232D307F232D307F232D307F232D3078
:100C80007F232D307F232D307F232D307F23023093
:100C9000BE000030A7222D307F232D307F232D3042
:100CA0007F230F307F233C307F2341307F2346302A
:100CB0007F234B307F2350307F230F30962EBE0191
:100CC000BE0A0030A7222D307F232D307F232D3008
:100CD0007F232D307F232D307F232D307F232D3018
:100CE0007F232D307F232D307F232D307F232D3008
:100CF0007F232D307F232D307F232D307F23023023
:100D0000BE000030A7222D307F232D307F232D30D1
:100D10007F232D307F232D307F230F307F233230F0
:100D20007F2337307F230F307F232D307F232D30DB
:100D30007F232D307F232D307F232D307F232303EE
:100D40000319BF2F2308023A0319872F8B13CC30C6
:100D5000C1238B172119B32E8B134430C1238B175A
:100D60002115AD0121122119051EBD2E211EBD2EFA
:100D70008B13BE30C1238B172114B122211CFD2CF3
:100D80008B132723A8002723AA008B17BC00280851
:100D90003F242112211121100430BE000030A7226F
:100DA0001430F200F3013108F1003008F000BE22E7
:100DB0007408BC007508BD00E2231430F200F30192
:100DC0003308F1003208F000BE227408BC00750838
:100DD000BD00E2231430F200F3013508F1003408BD
:100DE000F000BE227408BC007508BD00E223A5080F
:100DF000031D062FA408031D062FA608031D062F9A
:100E000039083804031D062FDC30072FF030BC00F2
:100E1000BD01E2231430F200F3013708F100360877
:100E2000F000BE227408BC007508BD00E223043047
:100E3000BC000130BD00E2231830BC000130BD0011
:100E4000E2230530BE000030A7221430F200F30187
:100E50003108F1003008F000BE220A307407BC00EF
:100E60000030031801307507BD00E2231430F20092
:100E7000F3013308F1003208F000BE220A30740793
:100E8000BC000030031801307507BD00E2231430A8
:100E9000F200F3013508F1003408F000BE220A30F8
:100EA0007407BC000030031801307507BD00E22351
:100EB000A508031D672FA408031D672FA608031D9F
:100EC000672F39083804031D672FE630682FFA3082
:100ED000BC00BD01E2231430F200F3013708F10039
:100EE0003608F000BE220A307407BC000030031838
:100EF00001307507BD00E2230E30BC000130BD009B
:100F0000E2232230BC000130BD00E223FD2C04307E
:100F1000BE000030A7222D307F232D307F232D30BF
:100F20007F232D307F232D307F232D307F232D30C5
:100F30007F232D307F232D307F232D307F232D30B5
:100F40007F232D307F232D307F232D307F230530CD
:100F5000BE000030A7222D307F232D307F232D307F
:100F60007F230F307F233C307F2341307F23463067
:100F70007F234B307F2350307F230F30F62F0430F8
:100F8000BE000030A7222D307F232D307F232D304F
:100F90007F232D307F232D307F232D307F232D3055
:100FA0007F232D307F232D307F232D307F232D3045
:100FB0007F232D307F232D307F232D307F2305305D
:100FC000BE000030A7222D307F232D307F232D300F
:100FD0007F232D307F232D307F230F307F2332302E
:100FE0007F2337307F230F307F232D307F232D3019
:100FF0007F232D307F232D307F232D307F23FD2C29
:02400E003C3F35
:00000001FF
